:020000040000FA
:020000000528D1
:08000800090021006830990095
:1000100023008C018E0124000F308C001F308E00D5
:10002000210007309500270020309200200000308A
:100030008B008C018E01A60121001F308C001F3027
:100040008E0024008C1520008C018E01A801A901CE
:10005000D830AA00A80A031D3328A90A031D332893
:10006000AA0A03193A28DF2000002108FF3A031DDD
:100070004E282A2824008C11210028308C008E0163
:10008000200010308C008E012700930120000830E2
:100090008B000C1A630000008B011928E820E8206F
:1000A000E820E820E820F9200021F9200021F920AB
:1000B0000021E820F92021186128A60A000000008C
:1000C00064280321F9200021E820F920A1186C28D8
:1000D000A60A000000006F280321F9200021E82073
:1000E000F920211A7728A60A000000007A280321A7
:1000F000F9200021E820F920A11A8228A60A000090
:10010000000085280321F9200021E820F920211B87
:100110008D28A60A0000000090280321F920002164
:10012000E820F920A11B9628A60A99280321F92086
:1001300002212608A700E820F9202718A328A60AEC
:1001400000000000A6280321F9200021E820F92062
:10015000A718AE28A60A00000000B1280321F92044
:100160000021E820F9202119B9280221E820F920EE
:10017000BD280321F920A60A0000A119C428000007
:1001800000000000E820C528A60A1030A607F920C4
:100190000321A60BC7282108A3006430A4002B303C
:1001A000A500DF2021082306031D4E28FF3021066D
:1001B00003192628A50BD128A40BCF284E280C08FC
:1001C0000F39A1000E080F39A200220EA10400343D
:1001D0000B30A0008E16FF208E12FF200221A00BF4
:1001E000EA2800008E16FF208E12FF20000000007B
:1001F00008004B30A0000000A00BFB280800000006
:080200000000000000000800EE
:020000040001F9
:02000E00A40D3F
:02001000FF1CD3
:00000001FF
